:1000000004C002C045C000C0189510EF18BB10EF27
:1000100017BB1EE312BB11E411BB12E019BF14E0C1
:1000200013BF112712BFC2E4829BCEE01127222703
:10003000969A2A95F1F72A95F1F72A95F1F72A95DC
:10004000F1F71A95B1F7969816B31F70E9F324D01B
:100050009923D1F3B92F17D01FD09B17A9F713D02D
:100060001BD09B1789F7492F4A95406B38D016B3A0
:100070001F70E9F708D010D09923C9F704D00CD02D
:100080009923A9F7E1CF772778947723F1F3F894B0
:100090000FB773950FBF189514E020E8992728BB78
:1000A0000000000000000000000000000000000050
:1000B000A6B3AF7031F4269593951A9581F79927D9
:1000C0000BC014E0AA0FAA0FAA0FAA0FAA0F18F0CC
:1000D0009C5F1A95D9F7939510EF18BB08956AE0C5
:1000E0004095089410F4909A02C09098000011D0A6
:1000F00010D046956A95B1F7089569E00AD009D005
:1001000008D08894819B08946A9511F05795F7CF91
:0A01100008953C2F3A95F1F7089589
:00000001FF
